:020000040000FA
:10000000831203138B0107309F00831603138113A0
:10001000EF3083160313860083120313073090001A
:1000200022140E1C22109A201720AD201028031035
:10003000A20DA30DA40DA50DA60DA70DA80DA90D2C
:10004000AA0DAB0DAC0DAD0DAE0DAF0DB00DB10DDC
:10005000B20DB30DB40DB50DB60DB70DB80DB90D8C
:10006000BA0DBB0DBC0DBD0DBE0DBF0DC00DC10D3C
:10007000C20DC30DC40DC50DC60DC70DC80DC90DEC
:10008000CA0DCB0DCC0DCD0DCE0DCF0DD00DD10D9C
:10009000D20DD30DD40DD50DD60DD70DD80DD90D4C
:1000A000DA0DDB0DDC0DDD0DDE0DDF0DE00D831651
:1000B0000313A00DA10DA20DA30DA40DA50DA60D5A
:1000C000A70DA80DA90DAA0DAB0DAC0DAD0DAE0D74
:1000D000AF0DB00DB10DB20DB30DB40DB50DB60D24
:1000E000B70DB80DB90DBA0DBB0DBC0DBD0DBE0DD4
:1000F000BF0DC00DC10DC20DC30DC40DC50DC60D84
:10010000C70DC80DC90DCA0DCB0DCC0DCD0DCE0D33
:10011000CF0DD00DD10DD20DD30DD40DD50DD60DE3
:10012000D70DD80DD90DDA0DDB0DDC0DDD0D8312E9
:100130000313080022080139A000003083160313BE
:10014000DD1B013083120313A0062018AA28A8285B
:10015000061608000000061208002130A100000069
:10016000000000000000000000000000A10BAF280C
:0E017000000000000000000000000000080079
:02400E00423F2F
:00000001FF
